:10E000008E00FFBDE750CE0000DFD0DFD7DFD58622
:10E010005397D97F00DB7F00DC7F00DDDFDE9FE0F0
:10E02000DFE286C097E4CEE667BDE54CCE55AAC6D2
:10E030006486058B05188155271F816E2714811072
:10E040002625CEFFFFEC018C00002714CEE6D34F2F
:10E05000201CCEE6DC86012015CEE6E58603200EE8
:10E06000CEE6EE86042007BDE55ACEE6C94F97DB23
:10E07000BDE54CCEE682BDE54CBDE59FCE00C0BD02
:10E08000E5E6BDE5F04D27EB814426037EE0BA814D
:10E090004726037EE1D6815326037EE209814C2682
:10E0A000037EE271815026037EE362815226037E65
:10E0B000E473CEE69FBDE54C20B908BDE5E6BDE5BD
:10E0C000FB5D2615BDE5E6A60026E796D18B809779
:10E0D000D396D0890097D2203896E697D196E597C7
:10E0E000D0BDE5E6A600812C27114D26C596D18B23
:10E0F0008097D396D0890097D2201608BDE5E6BD5B
:10E10000E5FBBDE5E65D27AA6D0026A6DEE508DF96
:10E11000D296D184F097E896D097E77F00D48D21EE
:10E12000BDE762261196D4810225F396D397D19646
:10E13000D297D07EE07396E897D196E797D07EE0AD
:10E140007396E7D6E8BDE557CEE6A7BDE54CCE0011
:10E15000C0DFE9C6108D295A26FBCEE6AABDE54CE4
:10E16000CE00C0C610A6000881202509817F2405A5
:10E17000BDE7672005862EBDE7675A26E87EE59550
:10E180008620BDE76796D4262596D091E726069689
:10E19000D191E827158620BDE767BDE767DEE9A7CF
:10E1A0000008DFE9DEE708DFE739860197D496D477
:10E1B000810126E1DEE7A60008DFE7DEE9A7000827
:10E1C000DFE9BDE55A96D291E7260A96D391E82673
:10E1D00004860297D43908BDE5E6BDE5FBA6002715
:10E1E000037EE0B25D2704DEE5DFE296E09AE127F8
:10E1F000029EE096E33696E23696DF3696DE369657
:10E20000DC3696DD3696E4363B08BDE5E6BDE5FB3B
:10E21000BDE5E66D0026575D2704DEE5DFD796D71E
:10E22000D6D8BDE557CEE6AABDE54CDED7A600BDE3
:10E23000E55A8620BDE767BDE59FCE00C0BDE5E697
:10E24000A6002607DED708DFD720D3812D2607DEDC
:10E25000D709DFD720C8812E26037EE073BDE5FBFA
:10E260005D270BDED796E6A70008DFD720B07EE05B
:10E27000B208BDE5E6BDE5FBBDE5E66D0026EFBDF8
:10E28000E759BDE5F08153276F813A270D810D27AE
:10E29000EE810A27EABDE75920F3BDE56F97EB163B
:10E2A000BDE56F97E79BEB97EBBDE56F97E89BEBC1
:10E2B00097EB96E89BE697E896E799E597E7DEE720
:10E2C000BDE56F97DA9BEB97EB5D2714BDE56F36E5
:10E2D0009BEB97EB327D00DA2603A700085A26EC69
:10E2E000BDE56F9BEB26087D00DA27A97EE073CEA3
:10E2F000E685BDE54C7EE073BDE75997DABDE56F75
:10E300001697EBBDE56F97E79BEB97EBBDE56F9736
:10E31000E89BEB97EB96E89BE697E896E799E597FD
:10E32000E7DEE7C0032718BDE56F369BEB97EB965A
:10E33000DA8131260632A700082001325A26E8BDCC
:10E34000E56F9BEB81FF261196DA81372711813823
:10E35000270D813927097EE295CEE692BDE54C7EF8
:10E36000E07308A600BDE5F0814927048153260328
:10E370000897D9BDE5E6BDE5FB5D272296E597E95F
:10E3800096E697EABDE5E6A600812C261108BDE5D4
:10E39000E6BDE5FB5D2707BDE5E66D0027037EE0F2
:10E3A000B2DEE508DFE596E690EA97E696E592E9C3
:10E3B00097E5DEE98D1E96E59AE626F896D981491D
:10E3C0002609CEE6AEBDE54C7EE073CEE6BCBDE5EB
:10E3D0004C7EE073C6107D00E5260696E61124010A
:10E3E0001696E61097E696E5820097E596D981495C
:10E3F000263F863ABDE76717BDE55AD7EBDFE996BA
:10E40000E9BDE55A96E99BEB97EB96EABDE55A968E
:10E41000EA9BEB97EB4FBDE55AA60036BDE55A32B5
:10E420009BEB97EB085A26F196EB40BDE55A7EE54B
:10E43000958653BDE7678631BDE767178B0397EB7A
:10E44000BDE55ADFE996E9BDE55A96E99BEB97EB06
:10E4500096EABDE55A96EA9BEB97EBA60036BDE53A
:10E460005A329BEB97EB085A26F196EB43BDE55ADF
:10E470007EE59508BDE5E6BDE5F04D2606BDE50166
:10E480007EE073DFE7CEE7186D002772A100270852
:10E4900008080808080820F0DFE9DEE708BDE5E61F
:10E4A0006D00265ADEE9EE04BDE54C863DBDE7670A
:10E4B000DEE9E601EE02C1012607A600BDE55A200D
:10E4C0000AA600BDE55AA601BDE55A8620BDE7674C
:10E4D000BDE59FCE00C0BDE5E6A600271EBDE5FB5D
:10E4E0005D271BDEE9E601EE02C101260696E6A7DE
:10E4F00000200896E5A70096E6A7017EE0737EE07F
:10E50000B2CEE6FDBDE54C96DCBDE55ACEE700BDDA
:10E51000E54C96DDBDE55ACEE704BDE54C96DED66A
:10E52000DFBDE557CEE708BDE54C96E0D6E1BDE599
:10E5300057CEE70DBDE54C96E2D6E3BDE557CEE7F5
:10E5400012BDE54C96E4BDE55A7EE595A60027068A
:10E55000BDE7670820F6398D011736444444448DE1
:10E560000132840F8B30813A25028B077EE7674F9B
:10E570008D04484848483716BDE759BDE5F081305D
:10E580002511813A250A8141250981472405800703
:10E5900080301B3339860DBDE767860A7EE767CE7C
:10E5A00000C05FBDE759810D2737810A27338108F5
:10E5B0002719817F2715812025E9818024E5C10F56
:10E5C00024E15CA70008BDE76720D85D27D55A097C
:10E5D0008608BDE7678620BDE7678608BDE7672038
:10E5E000C28DB26F0039A600812026030820F739BA
:10E5F00081612506817B24028BE0395F7F00E57F06
:10E6000000E6A6008DEA81302534813A250A814151
:10E61000252C814724288007803049494949497978
:10E6200000E67900E5497900E67900E5497900E6F8
:10E630007900E5497900E67900E5085C20C439CE27
:10E64000E6F7BDE54C3297E43297DD3297DC32973E
:10E65000DE3297DF3233C001D7E3820097E29FE0DA
:10E66000BDE5017EE0733B0D0A556E6976657273F8
:10E67000616C204D6F6E69746F7220363830300DCA
:10E680000A005D20004572726F7220696865780D1E
:10E690000A004572726F7220737265630D0A00453D
:10E6A00072726F720D0A00203A00203A20003A3050
:10E6B0003030303030303146460D0A005339303377
:10E6C0003030303046430D0A00556E6B6E6F776EFA
:10E6D0000D0A004D43363830300D0A004D433638B0
:10E6E00030310D0A004844363330310D0A004D42B6
:10E6F000383836310D0A005357490D0A00413D00A4
:10E7000020423D0020583D002053503D0020504302
:10E710003D00204343523D00410100DCE7404201FF
:10E7200000DDE742580200DEE744530200E0E7461E
:10E73000500200E0E749430100E4E74C000000001C
:10E7400041004200580053500050430043435200E0
:10E7500086059710860A9711399611848027FA96B4
:10E7600012399611848039369611842027FA32970F
:02E7700013395B
:03FF80007EE00020
:03FF88007EE073A5
:03FF90007EE767A2
:03FF98007EE54CB7
:03FFA0007EE759A0
:03FFA8007EE7628F
:08FFF800E666E63FE666E00064
:00000001FF
